:1000000092C0ACC05FC2AAC0A9C0A8C0A7C0A6C009
:10001000A5C0A4C0A3C0A2C0A1C0A0C09FC09EC0D4
:100020009DC09CC09BC004030904240368006100B8
:10003000660074006D0061006E006E0023007300A6
:100040006F006600740077006100720065003A037B
:100050005500530042002000460069006E00670012
:1000600065007200740069007000200043006F009A
:100070006E007400610063007400200047006C0093
:100080006F00760065007300120110010200000885
:10009000C016E10501460102000109024300020108
:1000A00000800A090400000102020100052400107A
:1000B00001042402020524060001052401030107AE
:1000C00005830308000209040100020A000000077A
:1000D0000501020800000705810208000056332EC2
:1000E00030422050494E43482062792046616B657A
:1000F000737061636520496E632E20313939352074
:100100002D20686166746D616E6E23736F667477FF
:100110006172650020474C4F564500204E4F2047E6
:100120004C4F5645000011241FBECFE5D4E0DEBF82
:10013000CDBF10E0A0E6B0E0EAE7F0E102C0059034
:100140000D92AE36B107D9F712E0AEE6B0E001C0CD
:100150001D92AB32B107E1F7BCD48EC751CF85B742
:10016000886085BF8BB780688BBF8BE48093FE006F
:100170008093F30008951F93DC01162F8091630094
:1001800084FF07C08091F30098E889278093F300EB
:1001900003C08AE580936300912FE4EFF0E002C092
:1001A0008D9181939150E0F7612F84EF90E086D19B
:1001B0001C5F109363001F9108951F93DC01162F9D
:1001C0008091620084FF07C08091FE0098E8892733
:1001D0008093FE0003C08AE580936200912FEFEFC9
:1001E000F0E002C08D9181939150E0F7612F8FEF85
:1001F00090E064D11C5F109362001F9108950F93EB
:100200001F93CF93DF9360910F0116160CF0C6C0B9
:10021000162F135080910B01CFE1D1E0C81BD109FB
:1002200080910A018D3211F48AEFBCD280910A01CB
:10023000803120F4612FCE0171D6AAC08D3209F031
:100240008CC08AE580936100183009F09BC08881DA
:10025000807609F06FC021EF30E01092F1008981C3
:10026000882341F41092F20030930E0120930D0187
:1002700092E06AC0853021F48A8180931001F5C034
:100280008630C1F58B81813041F488E890E090930D
:100290000E0180930D0192E1EBC0823041F48AE9B6
:1002A00090E090930E0180930D0193E4E1C08330C0
:1002B00009F0DDC08A81882341F486E290E09093C2
:1002C0000E0180930D0194E0D3C0813041F48AE2A5
:1002D00090E090930E0180930D0194E2C9C08230AA
:1002E00009F0C5C08EE490E090930E0180930D015B
:1002F0009AE3BEC0883039F482E191E090930E0118
:1003000080930D010CC0893021F48A818093120101
:10031000ACC08A3031F430930E0120930D0191E08E
:1003200013C08B3009F0A1C08BE48093FE00809352
:10033000F3009BC0CE0166D3982F8F3F29F48881AC
:1003400087FF1AC09E8118C020E88F818823E1F4BE
:100350008E818917C8F4982F17C080916E0087FD91
:1003600011C0612FCE01B7D58F3F41F4809360005B
:100370008EE1809361009FEF20E006C08823D9F3CF
:1003800090E0FACF90E020E820936E009093600018
:1003900080910F01181614F410920F0180916100E2
:1003A00084FF58C0809160008F3F09F453C0682FCC
:1003B000893008F068E0861B8093600080916E00B1
:1003C00080FF02C003EC01C00BE48F5F80936E00DE
:1003D00087FF23C020910D0130910E0186FD05C0DD
:1003E000962FF901A9EEB0E00DC0962FF901A9EE04
:1003F000B0E003C084918D9331969150D8F704C03A
:1004000081918D939150E0F7C901860F911D9093D2
:100410000E0180930D01772707C0662359F189EEFD
:1004200090E069D5682F7727162F693058F489EE48
:1004300090E044D0912F9C5F183040F48FEF809370
:10044000600004C08FEF809360009EE10093E8009D
:10045000909361009AE080B38C7091F49150D9F739
:1004600010921001109209010BC090E06DCF90E046
:1004700020EC6BCF60E089EE90E020D094E0DECFFE
:10048000DF91CF911F910F910895A82FB92F8FEF72
:100490009FEF41E050EA615070F02D9138E0722FEB
:1004A000782796958795269570FF02C08427952713
:1004B0003A95A9F7F0CF809590950895E6DF8D9352
:1004C0009D930895CF93CFB7CF93839BFECF839B0C
:1004D0000EC0839B0CC0839B0AC0839B08C0839B78
:1004E00006C0C0910C01C395C0930C01A6C0DF9358
:1004F000C0910B01DD27CD5EDE4F839B02C0DF91F3
:10050000E6CF2F930F931F9300B32FEF03FB20F938
:100510004F933F9310B34FEF012703FB21F93BE0CB
:1005200031C04E7F012F10B3216028C0102F4D7FA6
:100530002260000000B329C04B7F2460012F00001F
:1005400010B32BC010B3477F28602AC04F7E00B382
:1005500020612CC04F7D10B320622FC04F7B00B3B1
:10056000206432C0422700B349934FEF00001027A8
:1005700013FB20F910B31C70C9F1297F91F20127F8
:1005800003FB21F900B3237F89F2315058F1102782
:1005900013FB22F910B3277E79F2012703FB23F91D
:1005A0002F7C81F200B3102713FB24F92F7971F20D
:1005B00000C010B3012703FB25F92F7359F200C0C7
:1005C00000B3102713FB26F9223040F200C010B30D
:1005D000012703FB27F9243028F64F77206810B352
:1005E0000000F9CF10E81ABF00271CC03B5031951E
:1005F000C31BD04010E81ABF0881033C11F10B3433
:1006000001F1209109011981110F1213EDCF4A81D7
:10061000441F093659F10D3211F0013E29F74F7090
:1006200009F0042F009311013F914F911F910F91F9
:100630002F91DF91CAB7C7FD48CFCF91CFBFCF91E0
:10064000189500911101002379F310910F011123E6
:10065000F9F53430FAF130930F0100930A0110914B
:100660000B013BE0311B30930B0134C000910F01B3
:10067000013074F50AE54F7049F43091610034FDA2
:100680002BC000936100C8EED0E02AC0433049F08F
:100690003091620034FD20C000936200CEEFD0E0C4
:1006A0001FC03091630034FD17C000936300C3EF97
:1006B000D0E016C0052710E002BB1FC0052722C0EE
:1006C000052727C005272CC0052710E002BB33C033
:1006D0004AE503C042ED01C0432FC4E1D0E032E05F
:1006E00011B31C60939A02B311BB5F935CE020E8E6
:1006F00020FF052702BB279517951C3FD8F620FF42
:100700000527279502BB17951C3FC0F620FF05273C
:100710002795179502BB1C3F98F620FF05272795C4
:1007200017951C3F02BB70F600C0499120FF0527BA
:1007300002BB279517951C3F38F620FF0527279504
:1007400002BB17951C3F40F520FF052727951795FD
:1007500002BB1C3F18F520FF0527279517951C3F66
:1007600002BBF0F4242F3A9519F6037F5F9102BB88
:10077000000010911001110FC651D04011F01093DC
:10078000090110E81ABF086011B3137F402F437F9F
:1007900002BB11BB42BB48CF0527D2CF0527D7CF1D
:1007A0000527DCCF982F80917A00882319F4909345
:1007B0007C00AD9A90937B0090937A000895492F26
:1007C000552724B32F6124BB21B3206F21BBB89AD6
:1007D00025B38F712F61382F3095232325BB22B38A
:1007E000642F6295607F206F362F3095232322BBC4
:1007F00028B342954F7041702160342F30952323E8
:1008000028BB24B3207E282B24BB81B38F70862B7A
:1008100081BB87B38E7F842B87BB089523B3822F40
:10082000806E30B326B332953F702E6F2295207FB5
:10083000922F932B809590950895332019F0C298AC
:10084000BA9A08959098889A0895332019F0C29A18
:10085000BA980895909A88980895332019F0C1980D
:10086000B99A08959198899A0895332019F0C19AF8
:10087000B9980895919A89980895CF93DF93E5DF09
:10088000000000000000000000000000332011F014
:1008900086B301C080B3C82FDD27C270D070CDDF12
:1008A000CE01DF91CF9108950F931F93182F08E089
:1008B00017FF02C0DADF01C0D0DFDFDF015011F027
:1008C000110FF6CFD2DFD9DF99271F910F9108952D
:1008D000000000000000B9DF000000000000BDDFE4
:1008E000000000000000A9DF000000000000BDDFE4
:1008F0000895EF92FF920F931F93CF93DF93182FDA
:10090000EB01E42EE5DF80EACFDF8823E1F4812FDD
:10091000CBDF8823C1F4DCDF81EAC6DF882399F4CA
:10092000FF240DC018E000E0000FA7DF8111016077
:100930001150D1F7EF1091DFA0DF97DF0993F39407
:10094000EF1480F701C0FF2488DF000000000000E2
:100950007CDF00000000000088DF8F2D9927DF91E9
:10096000CF911F910F91FF90EF900895CF93DF9358
:10097000CDB7DEB721970FB6F894DEBF0FBECDBF5F
:100980001982232D332011F086B301C080B399273B
:1009900082709070882311F48CE40EC0222329F019
:1009A00086B399278470907004C080B399278170B2
:1009B0009070882319F482E5898306C041E0BE0166
:1009C0006F5F7F4F80E095DF8981992721960FB671
:1009D000F894DEBF0FBECDBFDF91CF9108953324D1
:1009E0002224C4DF682E3394C1DF782E962D9235F1
:1009F00019F4823529F408958C3419F49C3409F0E3
:100A000023940895FC012081822F80768032D9F4CE
:100A10009181892F8052823028F490939E008FEF2D
:100A200090E00895923239F48091A600882319F459
:100A300082E08093A60027FD06C088E08093A7008F
:100A400080E090E0089580E090E00895DC01662366
:100A5000C1F08091290190912A01891B815086174C
:100A600018F4862F9927089580912A01E82FFF27EF
:100A7000E75DFE4F9D9192838F5F80932A016150C5
:100A800099F780E090E00895AC01DC010AC0E22F04
:100A9000FF27E75DFE4F82818D932F5F2093290111
:100AA00061509A2F941B2091290180912A012817C7
:100AB00011F0662361F7892F99270895DC01D4D2BC
:100AC000802D681729F06DBBF894E29AE19A78942A
:100AD000089594B714BE479A88E10FB6F89481BD83
:100AE00011BC0FBE93FF0AC080B38C7039F080E850
:100AF0008BBF80EA85BF78948895F89480E885BF9D
:100B000088E190E028E00FB6F894A89581BD0FBE6B
:100B100021BD25DB78948FE385BB85B388BB83EF4C
:100B200082BB80E284BB80E88093E50058DFA0E0D0
:100B3000B0E09AD2802D813019F481E88093E500ED
:100B4000A1E0B0E091D2802D813011F471E0572EF8
:100B5000FF2480B38C7009F08895D0900C011D2D76
:100B60001F1921F480B38C7009F4ACC1A89547DB40
:100B7000112309F46CC18091E6009091E700810F88
:100B8000911D9093E7008093E60096FF06C08FEFDB
:100B90009FE39093E7008093E60080917C00909122
:100BA0007A0020917B0030E2992349F0815021F4B2
:100BB00085B3832785BB822F915009F4AD981150DE
:100BC00099F780937C0090937A0010927D0026DE46
:100BD0009C01009749F0552039F081112062C9012C
:100BE0008070892B09F03062C90140E050E080FD3F
:100BF0005F5F4F5F403119F096958795F8CF52307F
:100C000048F030937F0020937E0080917D008F5FBD
:100C100080937D00E901C06ED06E01E010E0EE240B
:100C2000FF24C8018C239D23892B39F5C801C7DD1A
:100C300084E600008150E9F7F1DD9E0120953095B2
:100C400028233923C90180239123892BE9F1C80185
:100C50008095909582239323892B79F0C22BD32BF7
:100C600080917D00E82FFF27EE0FFF1FE358FF4F15
:100C7000328321838F5F80937D00000F111F0894C2
:100C8000E11CF11C20E1E216F10459F680E090E04D
:100C900096DD10917D00412F5527440F551F4F5F62
:100CA0005F4F68E870E08DE790E0C8D1892B79F05C
:100CB000A8E8B0E0EDE7F0E08BE001900D92815004
:100CC000E1F71AE0412EC2C010927D00E2CF842DE0
:100CD000442009F4BBC08150482E09F0B7C0F4C0CD
:100CE000E32FFF27EE0FFF1FE358FF4F4181528193
:100CF00020E00CC0E22FFF27EE0FFF1FED56FF4F45
:100D0000818192814817590789F02F5F261791F743
:100D100080916F00E82FFF27EE0FFF1FE159FF4F73
:100D2000528341838F5F80936F0071E03F5F311783
:100D3000B9F630E028C080916F00E82FFF27EE0F52
:100D4000FF1FE159FF4F528341838F5F80936F00F4
:100D500019C0E32FFF27EE0FFF1FED56FF4F418114
:100D6000528120E00CC0E22FFF27EE0FFF1FE35857
:100D7000FF4F8181928148175907E9F22F5F2117B0
:100D800091F771E03F5F361721F7772309F45EC0D2
:100D9000A3E9B0E0EFE6F0E08BE001900D92815026
:100DA000E1F7772309F452C08091E6009091E700C3
:100DB0008051974208F013DE00919300F090E50017
:100DC000F092A900002319F4AAEAB0E01CC0222086
:100DD00079F0E3E9F0E0AAEAB0E082818C938181C6
:100DE000ED018983129601503296002361F0F5CF10
:100DF000000F1127A80164E970E08AEA90E02BD186
:100E0000D801A655BF4F21E8F21689F48091E6007B
:100E10009091E700282F2F77FD012193880F892FCC
:100E2000881F990B9195ED018983DF0111968FE859
:100E30008D9389EA90E06A2F681B08DE882321F4ED
:100E40001092E7001092E60084E6ACDCFD2C809165
:100E5000620084FF11C068E089EA90E015DE082F87
:100E6000882321F48091A70083FF06C0602F89EAC0
:100E700090E0A3D90093A7008091630084FF13C082
:100E80008091A600882379F0823021F468E084E61E
:100E900090E003C062E08CE690E06DD98091A600FE
:100EA00081508093A600E19954CE6091E50060588E
:100EB00080E090E003DEE1994CCE652D81E090E08A
:100EC000FDDD47CE9CD9C3CF10926F006091930097
:100ED00030E070E02CCF9C0180919E00803241F484
:100EE000AFE9B0E0F90187E001900D928150E1F7A0
:100EF00081E090E008959C0180919E00813219F07C
:100F000080E090E00895F901AFE9B0E087E00D904E
:100F100001928150E1F787E090E00895FF920F93EE
:100F20001F93CF93DF93EC01F62E0091A800662368
:100F300009F477C086E936DC1991002339F4812F52
:100F400081528E3508F068C0012F66C082E8809318
:100F5000A9000334E9F51C3411F0123579F53FDDB1
:100F6000161511F433240FC0171519F4E1E03E2EC5
:100F70000AC01093AA006BE171E08BEA90E057D0B1
:100F8000E4EBF0E041C04EE16AEA70E080E0B1DC01
:100F9000982F882349F0EAEAF0E0819180528F355A
:100FA00060F5915089F1F9CF1093AA0064E171E0E6
:100FB0008BEA90E03CD0E1EBF0E026C01035F9F48C
:100FC0006DED70E08AEA90E032D0E0EEF0E01CC017
:100FD000073431F4812F8053823088F4582E0AC0B0
:100FE000043569F4812F8053823048F4105B1093EC
:100FF000E50010551093AA0005C0319705C08FE396
:101000008093AA00EBEAF0E08FE8819389EA90E010
:101010006E2F681B1BDD00E0FA9409F08DCF009362
:10102000A800DF91CF911F910F91FF900895FB01D0
:10103000DC0105900D920020E1F70895FB01DC0131
:1010400004C08D910190801921F441505040C8F79F
:10105000881B990B0895FB01DC0102C001900D92E1
:1010600041505040D8F70895E199FECFBFBBAEBBC9
:0A107000E09A11960DB20895FFCF2B
:0E107A00FF5A5A5AA120000000000200030095
:00000001FF
